:020000040000FA
:040000006A303A2800
:08000800A000030EA100831209
:100010008B1C32288B1031181428B11C3228643004
:10002000010203183128182800001628172818285C
:1000300019281A281B281C281D281E281F283110A3
:10004000B114A810031005190314AA0DA90DA80DC9
:10005000B00B322831152A08AF002908AE00280855
:10006000AD00B11081010B11210E8300A00E200EF6
:02007000090085
:0C007400203084008001840A6030040207
:10008000031C3C281230B00062228316FF2390002C
:10009000831283160C308505870183128501870141
:1000A000073099000030831691008312C830831600
:1000B0008100831231309000003083168C0083124F
:1000C00010308B00831600309B001C141A0883121A
:1000D000BC00851D6F233C1C7C28831610309B00C0
:1000E0001C141A088312BD00831630309B001C14A8
:1000F0001A088312C200F922831620309B001C14B8
:100100001A088312C1000130C1080319C10081011E
:100110008E018F010B118B100B108C018B179F2000
:100120003119B5204122B30B9D2803108519031402
:10013000B90DF03039020319D0210E238F28640045
:10014000311808000B1D08000B11B11031141230CA
:10015000B000051DB0283214831601138312080065
:100160003210831601178312080031110130B700D5
:100170008B132030370783169B001C141A08831238
:10018000A400A500C030A5061030370783169B00D9
:100190001C141A088312A3000030370783169B0033
:1001A0001C141A088312A2008B17321CDD282209A6
:1001B0000339A200A309A409A50922082D02031DE1
:1001C000CA2923082E02031DCA2924082F02031D51
:1001D000572901303702031DF4283C19F3283D1834
:1001E000F4283D143E14632202303702031DFF2819
:1001F0003C19FE28BD18FF28BD143E146A220330A6
:100200003702031D0A293C1909293D190A293D1500
:100210003E14712204303702031D15293C1914299C
:10022000BD191529BD153E14782205303702031D6E
:1002300020293C191F293D1A20293D163E147F22F2
:1002400006303702031D2B293C192A29BD1A2B29F8
:10025000BD163E14862207303702031D36293C198D
:1002600035293D1B36293D173E148D2208303702B3
:10027000031D41293C194029BD1B4129BD173E14CE
:10028000942209303702031D4C293C194B2942188E
:100290004C2942143E149B220A303702031D572971
:1002A0003C195629C2185729C2143E14A222250807
:1002B0002F02031DCA2901303702031D66293C198C
:1002C00065293D1C66293D103E14A92202303702E3
:1002D000031D71293C197029BD1C7129BD103E14E4
:1002E000AD2203303702031D7C293C197B293D1DBB
:1002F0007C293D113E14B12204303702031D8729A9
:100300003C198629BD1D8729BD113E14B522053033
:100310003702031D92293C1991293D1E92293D1255
:100320003E14B92206303702031D9D293C199C2931
:10033000BD1E9D29BD123E14BD2207303702031D8C
:10034000A8293C19A7293D1FA8293D133E14C12205
:1003500008303702031DB3293C19B229BD1FB32948
:10036000BD133E14C52209303702031DBE293C19B6
:10037000BD29421CBE2942103E14C9220A30370250
:10038000031DC9293C19C829C21CC929C2103E1421
:10039000CD22CA29B70A0B30370203180800B82843
:1003A0000130B600B300B400B500B7008501870185
:1003B000B1139F20B30B102A031085190314B90D34
:1003C000F03039020319372AB40B102A01303702F2
:1003D0000319D122023037020319D5220330370224
:1003E0000319D922043037020319DD220530370200
:1003F0000319E122063037020319E52207303702DC
:100400000319E922083037020319ED2209303702B7
:100410000319F1220A3037020319F5229630B4008D
:10042000311DD9293111321C1A2A2D090339AD0089
:10043000AE09AF092F1CB1132F1CD929B11BD92923
:100440002E18D929B1178B1320303707BB002F087E
:10045000BA004F2210303707BB002E08BA004F22D7
:1004600000303707BB002D08BA004F228B178501DB
:100470008701B70AB6010B303702031CD929F922CC
:1004800008003E1C08003E101030BB003D08BA00BA
:100490004F223030BB004208BA004F2208008B13B5
:1004A0003A0883161C159A003B089B0055309D00A6
:1004B000AA309D009C1464009C185B2A1C118312B6
:1004C0008B1708000800051640084107D0000F08E8
:1004D000D1000800851640084107D2000F08D3005C
:1004E0000800051440084107D4000F08D500080093
:1004F000851440084107D6000F08D700080087146C
:1005000040084107D8000F08D90008000715400827
:100510004107DA000F08DB00080007144008410714
:10052000DC000F08DD000800871640084107DE00E8
:100530000F08DF000800071640084107CC000F082D
:10054000CD000800871540084107CE000F08CF00F6
:10055000080005128E018F01080085128E018F019F
:10056000080005108E018F01080085108E018F0193
:10057000080087108E018F01080007118E018F017E
:10058000080007108E018F01080087128E018F016D
:10059000080007128E018F01080087118E018F015C
:1005A00008000508103A850008000508203A850073
:1005B00008000508013A850008000508023A850090
:1005C00008000708023A870008000708043A870075
:1005D00008000708013A870008000708203A87004A
:1005E00008000708103A870008000708083A870043
:1005F00008003D180516BD1885163D190514BD19CE
:1006000085143D1A8714BD1A07153D1B0714BD1B21
:10061000871642180716C218871508003C1D0800E7
:1006200050084002031D192B51080F02031C192BFF
:10063000051252084002031D222B53080F02031C0F
:10064000222B851254084002031D2B2B55080F0244
:10065000031C2B2B051056084002031D342B570892
:100660000F02031C342B851058084002031D3D2B3C
:1006700059080F02031C3D2B87105A084002031D26
:10068000462B5B080F02031C462B07115C08400237
:10069000031D4F2B5D080F02031C4F2B07105E0834
:1006A0004002031D582B5F080F02031C582B8712B2
:1006B0004C084002031D612B4D080F02031C612BE7
:1006C00007124E084002031D6A2B4F080F02031C3D
:1006D0006A2B87110C1C08000C10C00A0800B60118
:1006E000B301B4013C1C772BBC01BC147E2BBC1C99
:1006F0007C2BBC013C157E2BBC013C143C08B60095
:100700006400822B832B842B852B862BB41B051630
:10071000B41F0512B30B802BB40B802B0310B60C47
:10072000B608031D802B0030BB003C08BA004F22E6
:020730000800BF
:084000000900030002000600A4
:02400E00CC01E3
:10420000010003000300030003000200020002009B
:1042100002000000000000000000FF00FF00FF009F
:10422000000000000000000000000000000000008E
:104230000000C000C000C000C000FF00FF00FF0081
:104240000100C300F300CF00FF00C300F300CF0064
:10425000FF00C300F300CF00FF00FF00FF00FF00DE
:10426000FF00FF00FF00FF00FF00FF00FF00FF0056
:10427000FF00FF00FF00FF00FF00FF00FF00FF0046
:10428000FF00FF00FF00FF00FF00FF00FF00FF0036
:10429000FF00FF00FF00FF00FF00FF00FF00FF0026
:1042A000FF00FF00FF00FF00FF00FF00FF00FF0016
:1042B000FF00FF00FF00FF00FF00FF00FF00FF0006
:1042C000FF00FF00FF00FF00FF00FF00FF00FF00F6
:1042D000FF00FF00FF00FF00FF00FF00FF00FF00E6
:1042E000FF00FF00FF00FF00FF00FF00FF00FF00D6
:1042F000FF00FF00FF00FF00FF00FF00FF00AA001B
:00000001FF
